 le

 Timestamp is 70a80123 (reproducible build file hash)

 Preferred load address is 0000000180000000

 Start         Length     Name                   Class
 0001:00000000 00002c70H .text$mn                CODE
 0001:00002c70 00000036H .text$mn$00             CODE
 0001:00002ca6 00000092H .text$x                 CODE
 0002:00000000 00000198H .idata$5                DATA
 0002:00000198 00000038H .00cfg                  DATA
 0002:000001d0 00000008H .CRT$XCA                DATA
 0002:000001d8 00000008H .CRT$XCZ                DATA
 0002:000001e0 00000008H .CRT$XIA                DATA
 0002:000001e8 00000008H .CRT$XIZ                DATA
 0002:000001f0 00000008H .CRT$XPA                DATA
 0002:000001f8 00000008H .CRT$XPZ                DATA
 0002:00000200 00000008H .CRT$XTA                DATA
 0002:00000208 00000008H .CRT$XTZ                DATA
 0002:00000210 00000000H .gehcont$y              DATA
 0002:00000210 00000000H .gfids$y                DATA
 0002:00000210 00000bf0H .rdata                  DATA
 0002:00000e00 00000000H .rdata$CastGuardVftablesA DATA
 0002:00000e00 00000000H .rdata$CastGuardVftablesC DATA
 0002:00000e00 000001f4H .rdata$r                DATA
 0002:00000ff4 00000064H .rdata$voltmd           DATA
 0002:00001058 00000300H .rdata$zzzdbg           DATA
 0002:00001358 00000008H .rtc$IAA                DATA
 0002:00001360 00000008H .rtc$IZZ                DATA
 0002:00001368 00000008H .rtc$TAA                DATA
 0002:00001370 00000008H .rtc$TZZ                DATA
 0002:00001378 00000240H .xdata                  DATA
 0002:000015b8 000000f8H .xdata$x                DATA
 0002:000016b0 00000540H .edata                  DATA
 0002:00001bf0 00000050H .idata$2                DATA
 0002:00001c40 00000018H .idata$3                DATA
 0002:00001c58 00000198H .idata$4                DATA
 0002:00001df0 00000460H .idata$6                DATA
 0003:00000000 00000038H .data                   DATA
 0003:00000038 00000080H .data$r                 DATA
 0003:000000b8 00000028H .data$rs                DATA
 0003:000000e0 00000818H .bss                    DATA
 0004:00000000 000002d0H .pdata                  DATA
 0005:00000000 00000060H .rsrc$01                DATA
 0005:00000060 00000300H .rsrc$02                DATA

  Address         Publics by Value              Rva+Base               Lib:Object

 0000:00000000       __AbsoluteZero             0000000000000000     <absolute>
 0000:00000000       ___safe_se_handler_count   0000000000000000     <absolute>
 0000:00000000       ___safe_se_handler_table   0000000000000000     <absolute>
 0000:00000000       __arm64x_extra_rfe_table   0000000000000000     <absolute>
 0000:00000000       __arm64x_extra_rfe_table_size 0000000000000000     <absolute>
 0000:00000000       __arm64x_native_entrypoint 0000000000000000     <absolute>
 0000:00000000       __arm64x_redirection_metadata 0000000000000000     <absolute>
 0000:00000000       __arm64x_redirection_metadata_count 0000000000000000     <absolute>
 0000:00000000       __dynamic_value_reloc_table 0000000000000000     <absolute>
 0000:00000000       __enclave_config           0000000000000000     <absolute>
 0000:00000000       __guard_check_icall_a64n_fptr 0000000000000000     <absolute>
 0000:00000000       __guard_eh_cont_count      0000000000000000     <absolute>
 0000:00000000       __guard_eh_cont_table      0000000000000000     <absolute>
 0000:00000000       __guard_fids_count         0000000000000000     <absolute>
 0000:00000000       __guard_fids_table         0000000000000000     <absolute>
 0000:00000000       __guard_iat_count          0000000000000000     <absolute>
 0000:00000000       __guard_iat_table          0000000000000000     <absolute>
 0000:00000000       __guard_longjmp_count      0000000000000000     <absolute>
 0000:00000000       __guard_longjmp_table      0000000000000000     <absolute>
 0000:00000000       __hybrid_auxiliary_delayload_iat 0000000000000000     <absolute>
 0000:00000000       __hybrid_auxiliary_delayload_iat_copy 0000000000000000     <absolute>
 0000:00000000       __hybrid_auxiliary_iat     0000000000000000     <absolute>
 0000:00000000       __hybrid_auxiliary_iat_copy 0000000000000000     <absolute>
 0000:00000000       __hybrid_code_map          0000000000000000     <absolute>
 0000:00000000       __hybrid_code_map_count    0000000000000000     <absolute>
 0000:00000000       __hybrid_image_info_bitfield 0000000000000000     <absolute>
 0000:00000000       __x64_code_ranges_to_entry_points 0000000000000000     <absolute>
 0000:00000000       __x64_code_ranges_to_entry_points_count 0000000000000000     <absolute>
 0000:00000100       __guard_flags              0000000000000100     <absolute>
 0000:00000000       __ImageBase                0000000180000000     <linker-defined>
 0001:00000000       ?NewObject@JNIEnv_@@QEAAPEAV_jobject@@PEAV_jclass@@PEAU_jmethodID@@ZZ 0000000180001000 f i Kernel32.obj
 0001:00000024       Java_jdk_internal_org_jline_terminal_impl_jna_win_Kernel32Impl_FillConsoleOutputAttribute 0000000180001024 f   Kernel32.obj
 0001:00000118       Java_jdk_internal_org_jline_terminal_impl_jna_win_Kernel32Impl_FillConsoleOutputCharacter 0000000180001118 f   Kernel32.obj
 0001:0000020c       Java_jdk_internal_org_jline_terminal_impl_jna_win_Kernel32Impl_GetConsoleMode 000000018000120c f   Kernel32.obj
 0001:000002a0       Java_jdk_internal_org_jline_terminal_impl_jna_win_Kernel32Impl_GetConsoleScreenBufferInfo 00000001800012a0 f   Kernel32.obj
 0001:00000538       Java_jdk_internal_org_jline_terminal_impl_jna_win_Kernel32Impl_GetStdHandle 0000000180001538 f   Kernel32.obj
 0001:00000550       Java_jdk_internal_org_jline_terminal_impl_jna_win_Kernel32Impl_ReadConsoleInput 0000000180001550 f   Kernel32.obj
 0001:00000a84       Java_jdk_internal_org_jline_terminal_impl_jna_win_Kernel32Impl_ScrollConsoleScreenBuffer 0000000180001a84 f   Kernel32.obj
 0001:00000c7c       Java_jdk_internal_org_jline_terminal_impl_jna_win_Kernel32Impl_SetConsoleCursorPosition 0000000180001c7c f   Kernel32.obj
 0001:00000d34       Java_jdk_internal_org_jline_terminal_impl_jna_win_Kernel32Impl_SetConsoleMode 0000000180001d34 f   Kernel32.obj
 0001:00000da8       Java_jdk_internal_org_jline_terminal_impl_jna_win_Kernel32Impl_SetConsoleTextAttribute 0000000180001da8 f   Kernel32.obj
 0001:00000e1c       Java_jdk_internal_org_jline_terminal_impl_jna_win_Kernel32Impl_SetConsoleTitle 0000000180001e1c f   Kernel32.obj
 0001:00000ea8       Java_jdk_internal_org_jline_terminal_impl_jna_win_Kernel32Impl_WaitForSingleObject 0000000180001ea8 f   Kernel32.obj
 0001:00000ee0       Java_jdk_internal_org_jline_terminal_impl_jna_win_Kernel32Impl_WriteConsoleW 0000000180001ee0 f   Kernel32.obj
 0001:00000ff0       Java_jdk_internal_org_jline_terminal_impl_jna_win_Kernel32Impl_initIDs 0000000180001ff0 f   Kernel32.obj
 0001:00001c58       ??3@YAXPEAX_K@Z            0000000180002c58 f   MSVCRT:delete_scalar_size.obj
 0001:00001c60       ??_U@YAPEAX_K@Z            0000000180002c60 f   MSVCRT:new_array.obj
 0001:00001c68       __GSHandlerCheck           0000000180002c68 f   MSVCRT:gshandler.obj
 0001:00001c88       __GSHandlerCheckCommon     0000000180002c88 f   MSVCRT:gshandler.obj
 0001:00001d00       __security_check_cookie    0000000180002d00 f   MSVCRT:amdsecgs.obj
 0001:00002040       _DllMainCRTStartup         0000000180003040 f   MSVCRT:dll_dllmain.obj
 0001:00002080       ??3@YAXPEAX@Z              0000000180003080 f   MSVCRT:delete_scalar.obj
 0001:00002088       ??2@YAPEAX_K@Z             0000000180003088 f   MSVCRT:new_scalar.obj
 0001:000020c4       __raise_securityfailure    00000001800030c4 f   MSVCRT:gs_report.obj
 0001:000020f8       __report_gsfailure         00000001800030f8 f   MSVCRT:gs_report.obj
 0001:00002240       __security_init_cookie     0000000180003240 f   MSVCRT:gs_support.obj
 0001:000022ec       DllMain                    00000001800032ec f   MSVCRT:dll_dllmain_stub.obj
 0001:00002310       ?__scrt_initialize_type_info@@YAXXZ 0000000180003310 f   MSVCRT:tncleanup.obj
 0001:00002320       ?__scrt_uninitialize_type_info@@YAXXZ 0000000180003320 f   MSVCRT:tncleanup.obj
 0001:0000232c       __local_stdio_printf_options 000000018000332c f i MSVCRT:default_local_stdio_options.obj
 0001:00002334       __local_stdio_scanf_options 0000000180003334 f i MSVCRT:default_local_stdio_options.obj
 0001:0000233c       __scrt_initialize_default_local_stdio_options 000000018000333c f   MSVCRT:default_local_stdio_options.obj
 0001:00002358       __scrt_acquire_startup_lock 0000000180003358 f   MSVCRT:utility.obj
 0001:00002394       __scrt_dllmain_after_initialize_c 0000000180003394 f   MSVCRT:utility.obj
 0001:000023c8       __scrt_dllmain_before_initialize_c 00000001800033c8 f   MSVCRT:utility.obj
 0001:000023e0       __scrt_dllmain_crt_thread_attach 00000001800033e0 f   MSVCRT:utility.obj
 0001:00002408       __scrt_dllmain_crt_thread_detach 0000000180003408 f   MSVCRT:utility.obj
 0001:00002420       __scrt_dllmain_exception_filter 0000000180003420 f   MSVCRT:utility.obj
 0001:00002480       __scrt_dllmain_uninitialize_c 0000000180003480 f   MSVCRT:utility.obj
 0001:000024b0       __scrt_dllmain_uninitialize_critical 00000001800034b0 f   MSVCRT:utility.obj
 0001:000024c4       __scrt_initialize_crt      00000001800034c4 f   MSVCRT:utility.obj
 0001:00002510       __scrt_initialize_onexit_tables 0000000180003510 f   MSVCRT:utility.obj
 0001:0000259c       __scrt_is_nonwritable_in_current_image 000000018000359c f   MSVCRT:utility.obj
 0001:00002634       __scrt_release_startup_lock 0000000180003634 f   MSVCRT:utility.obj
 0001:00002658       __scrt_uninitialize_crt    0000000180003658 f   MSVCRT:utility.obj
 0001:00002684       __scrt_get_dyn_tls_init_callback 0000000180003684 f   MSVCRT:dyn_tls_init.obj
 0001:0000268c       __crt_debugger_hook        000000018000368c f   MSVCRT:utility_desktop.obj
 0001:00002694       __scrt_fastfail            0000000180003694 f   MSVCRT:utility_desktop.obj
 0001:000027e0       _RTC_Initialize            00000001800037e0 f   MSVCRT:initsect.obj
 0001:0000281c       _RTC_Terminate             000000018000381c f   MSVCRT:initsect.obj
 0001:00002858       _guard_check_icall_nop     0000000180003858 f i MSVCRT:guard_support.obj
 0001:0000285c       ??0bad_alloc@std@@QEAA@AEBV01@@Z 000000018000385c f i MSVCRT:throw_bad_alloc.obj
 0001:00002898       ??0bad_alloc@std@@QEAA@XZ  0000000180003898 f i MSVCRT:throw_bad_alloc.obj
 0001:000028b8       ??0bad_array_new_length@std@@QEAA@AEBV01@@Z 00000001800038b8 f i MSVCRT:throw_bad_alloc.obj
 0001:000028f4       ??0bad_array_new_length@std@@QEAA@XZ 00000001800038f4 f i MSVCRT:throw_bad_alloc.obj
 0001:00002914       ??0exception@std@@QEAA@AEBV01@@Z 0000000180003914 f i MSVCRT:throw_bad_alloc.obj
 0001:00002948       ??1bad_alloc@std@@UEAA@XZ  0000000180003948 f i MSVCRT:throw_bad_alloc.obj
 0001:00002948       ??1bad_array_new_length@std@@UEAA@XZ 0000000180003948 f i MSVCRT:throw_bad_alloc.obj
 0001:0000295c       ??_Ebad_alloc@std@@UEAAPEAXI@Z 000000018000395c f i MSVCRT:throw_bad_alloc.obj
 0001:0000295c       ??_Ebad_array_new_length@std@@UEAAPEAXI@Z 000000018000395c f i MSVCRT:throw_bad_alloc.obj
 0001:0000295c       ??_Eexception@std@@UEAAPEAXI@Z 000000018000395c f i MSVCRT:throw_bad_alloc.obj
 0001:0000295c       ??_Gbad_alloc@std@@UEAAPEAXI@Z 000000018000395c f i MSVCRT:throw_bad_alloc.obj
 0001:0000295c       ??_Gbad_array_new_length@std@@UEAAPEAXI@Z 000000018000395c f i MSVCRT:throw_bad_alloc.obj
 0001:0000295c       ??_Gexception@std@@UEAAPEAXI@Z 000000018000395c f i MSVCRT:throw_bad_alloc.obj
 0001:000029a0       ?__scrt_throw_std_bad_alloc@@YAXXZ 00000001800039a0 f   MSVCRT:throw_bad_alloc.obj
 0001:000029c0       ?__scrt_throw_std_bad_array_new_length@@YAXXZ 00000001800039c0 f   MSVCRT:throw_bad_alloc.obj
 0001:000029e0       ?what@exception@std@@UEBAPEBDXZ 00000001800039e0 f i MSVCRT:throw_bad_alloc.obj
 0001:000029f4       __isa_available_init       00000001800039f4 f   MSVCRT:cpu_disp.obj
 0001:00002ba0       _get_startup_argv_mode     0000000180003ba0 f   MSVCRT:argv_mode.obj
 0001:00002ba8       __scrt_is_ucrt_dll_in_use  0000000180003ba8 f   MSVCRT:ucrt_detection.obj
 0001:00002bc0       ??_Etype_info@@UEAAPEAXI@Z 0000000180003bc0 f i MSVCRT:std_type_info_static.obj
 0001:00002bc0       ??_Gtype_info@@UEAAPEAXI@Z 0000000180003bc0 f i MSVCRT:std_type_info_static.obj
 0001:00002beb       __C_specific_handler       0000000180003beb f   vcruntime:VCRUNTIME140.dll
 0001:00002bf1       __std_type_info_destroy_list 0000000180003bf1 f   vcruntime:VCRUNTIME140.dll
 0001:00002bf7       memset                     0000000180003bf7 f   vcruntime:VCRUNTIME140.dll
 0001:00002bfd       __std_exception_copy       0000000180003bfd f   vcruntime:VCRUNTIME140.dll
 0001:00002c03       __std_exception_destroy    0000000180003c03 f   vcruntime:VCRUNTIME140.dll
 0001:00002c09       _CxxThrowException         0000000180003c09 f   vcruntime:VCRUNTIME140.dll
 0001:00002c0f       _initterm                  0000000180003c0f f   ucrt:api-ms-win-crt-runtime-l1-1-0.dll
 0001:00002c15       _initterm_e                0000000180003c15 f   ucrt:api-ms-win-crt-runtime-l1-1-0.dll
 0001:00002c1b       free                       0000000180003c1b f   ucrt:api-ms-win-crt-heap-l1-1-0.dll
 0001:00002c21       _callnewh                  0000000180003c21 f   ucrt:api-ms-win-crt-heap-l1-1-0.dll
 0001:00002c27       malloc                     0000000180003c27 f   ucrt:api-ms-win-crt-heap-l1-1-0.dll
 0001:00002c2d       _seh_filter_dll            0000000180003c2d f   ucrt:api-ms-win-crt-runtime-l1-1-0.dll
 0001:00002c33       _configure_narrow_argv     0000000180003c33 f   ucrt:api-ms-win-crt-runtime-l1-1-0.dll
 0001:00002c39       _initialize_narrow_environment 0000000180003c39 f   ucrt:api-ms-win-crt-runtime-l1-1-0.dll
 0001:00002c3f       _initialize_onexit_table   0000000180003c3f f   ucrt:api-ms-win-crt-runtime-l1-1-0.dll
 0001:00002c45       _execute_onexit_table      0000000180003c45 f   ucrt:api-ms-win-crt-runtime-l1-1-0.dll
 0001:00002c4b       _cexit                     0000000180003c4b f   ucrt:api-ms-win-crt-runtime-l1-1-0.dll
 0001:00002c54       __acrt_initialize          0000000180003c54 f   MSVCRT:ucrt_stubs.obj
 0001:00002c54       __acrt_thread_attach       0000000180003c54 f   MSVCRT:ucrt_stubs.obj
 0001:00002c54       __acrt_thread_detach       0000000180003c54 f   MSVCRT:ucrt_stubs.obj
 0001:00002c54       __acrt_uninitialize        0000000180003c54 f   MSVCRT:ucrt_stubs.obj
 0001:00002c54       __acrt_uninitialize_critical 0000000180003c54 f   MSVCRT:ucrt_stubs.obj
 0001:00002c54       __scrt_stub_for_acrt_initialize 0000000180003c54 f   MSVCRT:ucrt_stubs.obj
 0001:00002c54       __scrt_stub_for_acrt_thread_attach 0000000180003c54 f   MSVCRT:ucrt_stubs.obj
 0001:00002c54       __scrt_stub_for_acrt_thread_detach 0000000180003c54 f   MSVCRT:ucrt_stubs.obj
 0001:00002c54       __scrt_stub_for_acrt_uninitialize 0000000180003c54 f   MSVCRT:ucrt_stubs.obj
 0001:00002c54       __scrt_stub_for_acrt_uninitialize_critical 0000000180003c54 f   MSVCRT:ucrt_stubs.obj
 0001:00002c54       __vcrt_initialize          0000000180003c54 f   MSVCRT:ucrt_stubs.obj
 0001:00002c54       __vcrt_thread_attach       0000000180003c54 f   MSVCRT:ucrt_stubs.obj
 0001:00002c54       __vcrt_thread_detach       0000000180003c54 f   MSVCRT:ucrt_stubs.obj
 0001:00002c54       __vcrt_uninitialize        0000000180003c54 f   MSVCRT:ucrt_stubs.obj
 0001:00002c54       __vcrt_uninitialize_critical 0000000180003c54 f   MSVCRT:ucrt_stubs.obj
 0001:00002c58       __scrt_stub_for_is_c_termination_complete 0000000180003c58 f   MSVCRT:ucrt_stubs.obj
 0001:00002c58       _is_c_termination_complete 0000000180003c58 f   MSVCRT:ucrt_stubs.obj
 0001:00002c5b       memcpy                     0000000180003c5b f   vcruntime:VCRUNTIME140.dll
 0001:00002c80       _guard_dispatch_icall_nop  0000000180003c80 f   MSVCRT:guard_dispatch.obj
 0001:00002ca0       _guard_xfg_dispatch_icall_nop 0000000180003ca0 f   MSVCRT:guard_xfg_dispatch.obj
 0002:00000000       __imp_GetStdHandle         0000000180004000     kernel32:KERNEL32.dll
 0002:00000008       __imp_GetLastError         0000000180004008     kernel32:KERNEL32.dll
 0002:00000010       __imp_WaitForSingleObject  0000000180004010     kernel32:KERNEL32.dll
 0002:00000018       __imp_GetConsoleMode       0000000180004018     kernel32:KERNEL32.dll
 0002:00000020       __imp_SetConsoleMode       0000000180004020     kernel32:KERNEL32.dll
 0002:00000028       __imp_ReadConsoleInputW    0000000180004028     kernel32:KERNEL32.dll
 0002:00000030       __imp_WriteConsoleW        0000000180004030     kernel32:KERNEL32.dll
 0002:00000038       __imp_FillConsoleOutputCharacterA 0000000180004038     kernel32:KERNEL32.dll
 0002:00000040       __imp_FillConsoleOutputAttribute 0000000180004040     kernel32:KERNEL32.dll
 0002:00000048       __imp_GetConsoleScreenBufferInfo 0000000180004048     kernel32:KERNEL32.dll
 0002:00000050       __imp_SetConsoleCursorPosition 0000000180004050     kernel32:KERNEL32.dll
 0002:00000058       __imp_SetConsoleTextAttribute 0000000180004058     kernel32:KERNEL32.dll
 0002:00000060       __imp_ScrollConsoleScreenBufferA 0000000180004060     kernel32:KERNEL32.dll
 0002:00000068       __imp_SetConsoleTitleA     0000000180004068     kernel32:KERNEL32.dll
 0002:00000070       __imp_RtlCaptureContext    0000000180004070     kernel32:KERNEL32.dll
 0002:00000078       __imp_RtlLookupFunctionEntry 0000000180004078     kernel32:KERNEL32.dll
 0002:00000080       __imp_RtlVirtualUnwind     0000000180004080     kernel32:KERNEL32.dll
 0002:00000088       __imp_UnhandledExceptionFilter 0000000180004088     kernel32:KERNEL32.dll
 0002:00000090       __imp_SetUnhandledExceptionFilter 0000000180004090     kernel32:KERNEL32.dll
 0002:00000098       __imp_GetCurrentProcess    0000000180004098     kernel32:KERNEL32.dll
 0002:000000a0       __imp_TerminateProcess     00000001800040a0     kernel32:KERNEL32.dll
 0002:000000a8       __imp_IsProcessorFeaturePresent 00000001800040a8     kernel32:KERNEL32.dll
 0002:000000b0       __imp_QueryPerformanceCounter 00000001800040b0     kernel32:KERNEL32.dll
 0002:000000b8       __imp_GetCurrentProcessId  00000001800040b8     kernel32:KERNEL32.dll
 0002:000000c0       __imp_GetCurrentThreadId   00000001800040c0     kernel32:KERNEL32.dll
 0002:000000c8       __imp_GetSystemTimeAsFileTime 00000001800040c8     kernel32:KERNEL32.dll
 0002:000000d0       __imp_DisableThreadLibraryCalls 00000001800040d0     kernel32:KERNEL32.dll
 0002:000000d8       __imp_InitializeSListHead  00000001800040d8     kernel32:KERNEL32.dll
 0002:000000e0       __imp_IsDebuggerPresent    00000001800040e0     kernel32:KERNEL32.dll
 0002:000000e8       \177KERNEL32_NULL_THUNK_DATA 00000001800040e8     kernel32:KERNEL32.dll
 0002:000000f0       __imp___C_specific_handler 00000001800040f0     vcruntime:VCRUNTIME140.dll
 0002:000000f8       __imp___std_type_info_destroy_list 00000001800040f8     vcruntime:VCRUNTIME140.dll
 0002:00000100       __imp_memset               0000000180004100     vcruntime:VCRUNTIME140.dll
 0002:00000108       __imp___std_exception_copy 0000000180004108     vcruntime:VCRUNTIME140.dll
 0002:00000110       __imp___std_exception_destroy 0000000180004110     vcruntime:VCRUNTIME140.dll
 0002:00000118       __imp__CxxThrowException   0000000180004118     vcruntime:VCRUNTIME140.dll
 0002:00000120       __imp_memcpy               0000000180004120     vcruntime:VCRUNTIME140.dll
 0002:00000128       \177VCRUNTIME140_NULL_THUNK_DATA 0000000180004128     vcruntime:VCRUNTIME140.dll
 0002:00000130       __imp_free                 0000000180004130     ucrt:api-ms-win-crt-heap-l1-1-0.dll
 0002:00000138       __imp__callnewh            0000000180004138     ucrt:api-ms-win-crt-heap-l1-1-0.dll
 0002:00000140       __imp_malloc               0000000180004140     ucrt:api-ms-win-crt-heap-l1-1-0.dll
 0002:00000148       \177api-ms-win-crt-heap-l1-1-0_NULL_THUNK_DATA 0000000180004148     ucrt:api-ms-win-crt-heap-l1-1-0.dll
 0002:00000150       __imp__seh_filter_dll      0000000180004150     ucrt:api-ms-win-crt-runtime-l1-1-0.dll
 0002:00000158       __imp__configure_narrow_argv 0000000180004158     ucrt:api-ms-win-crt-runtime-l1-1-0.dll
 0002:00000160       __imp__initialize_narrow_environment 0000000180004160     ucrt:api-ms-win-crt-runtime-l1-1-0.dll
 0002:00000168       __imp__initterm_e          0000000180004168     ucrt:api-ms-win-crt-runtime-l1-1-0.dll
 0002:00000170       __imp__execute_onexit_table 0000000180004170     ucrt:api-ms-win-crt-runtime-l1-1-0.dll
 0002:00000178       __imp__cexit               0000000180004178     ucrt:api-ms-win-crt-runtime-l1-1-0.dll
 0002:00000180       __imp__initialize_onexit_table 0000000180004180     ucrt:api-ms-win-crt-runtime-l1-1-0.dll
 0002:00000188       __imp__initterm            0000000180004188     ucrt:api-ms-win-crt-runtime-l1-1-0.dll
 0002:00000190       \177api-ms-win-crt-runtime-l1-1-0_NULL_THUNK_DATA 0000000180004190     ucrt:api-ms-win-crt-runtime-l1-1-0.dll
 0002:00000198       __guard_check_icall_fptr   0000000180004198     MSVCRT:guard_support.obj
 0002:000001a0       __guard_xfg_check_icall_fptr 00000001800041a0     MSVCRT:guard_support.obj
 0002:000001a8       __guard_dispatch_icall_fptr 00000001800041a8     MSVCRT:guard_support.obj
 0002:000001b0       __guard_xfg_dispatch_icall_fptr 00000001800041b0     MSVCRT:guard_support.obj
 0002:000001b8       __guard_xfg_table_dispatch_icall_fptr 00000001800041b8     MSVCRT:guard_support.obj
 0002:000001c0       __castguard_check_failure_os_handled_fptr 00000001800041c0     MSVCRT:guard_support.obj
 0002:000001c8       __guard_memcpy_fptr        00000001800041c8     vcruntime:softmemtag.obj
 0002:000001d0       __xc_a                     00000001800041d0     MSVCRT:initializers.obj
 0002:000001d8       __xc_z                     00000001800041d8     MSVCRT:initializers.obj
 0002:000001e0       __xi_a                     00000001800041e0     MSVCRT:initializers.obj
 0002:000001e8       __xi_z                     00000001800041e8     MSVCRT:initializers.obj
 0002:000001f0       __xp_a                     00000001800041f0     MSVCRT:initializers.obj
 0002:000001f8       __xp_z                     00000001800041f8     MSVCRT:initializers.obj
 0002:00000200       __xt_a                     0000000180004200     MSVCRT:initializers.obj
 0002:00000208       __xt_z                     0000000180004208     MSVCRT:initializers.obj
 0002:00000210       ??_C@_0DF@LIHHLEHB@jdk?1internal?1org?1jline?1terminal@ 0000000180004210     Kernel32.obj
 0002:00000248       ??_C@_04OHLIFDMD@?$CIJ?$CJV@ 0000000180004248     Kernel32.obj
 0002:00000250       ??_C@_06FALKBLGB@?$DMinit?$DO@ 0000000180004250     Kernel32.obj
 0002:00000258       ??_C@_01LELAEKIP@J@        0000000180004258     Kernel32.obj
 0002:0000025c       ??_C@_05MFEJDJP@value@     000000018000425c     Kernel32.obj
 0002:00000270       ??_C@_0EA@DDCNJKJC@jdk?1internal?1org?1jline?1terminal@ 0000000180004270     Kernel32.obj
 0002:000002b0       ??_C@_0DM@MBLFOGAB@jdk?1internal?1org?1jline?1terminal@ 00000001800042b0     Kernel32.obj
 0002:000002ec       ??_C@_01JPJNBJEM@I@        00000001800042ec     Kernel32.obj
 0002:000002f0       ??_C@_0EA@EMLEKAEK@jdk?1internal?1org?1jline?1terminal@ 00000001800042f0     Kernel32.obj
 0002:00000330       ??_C@_03GAEACAIP@?$CI?$CJV@ 0000000180004330     Kernel32.obj
 0002:00000340       ??_C@_0EC@GLHGKIHD@Ljdk?1internal?1org?1jline?1termina@ 0000000180004340     Kernel32.obj
 0002:00000384       ??_C@_05KAAPIFDI@uChar@    0000000180004384     Kernel32.obj
 0002:0000038c       ??_C@_01CPLAODJH@S@        000000018000438c     Kernel32.obj
 0002:00000390       ??_C@_0L@PLFFHFAH@Attributes@ 0000000180004390     Kernel32.obj
 0002:000003a0       ??_C@_0EK@EAOKBDCN@jdk?1internal?1org?1jline?1terminal@ 00000001800043a0     Kernel32.obj
 0002:000003ec       ??_C@_06HDDMAKPI@dwSize@   00000001800043ec     Kernel32.obj
 0002:000003f4       ??_C@_01POHCFINO@Z@        00000001800043f4     Kernel32.obj
 0002:000003f8       ??_C@_08DHPIEJHJ@bVisible@ 00000001800043f8     Kernel32.obj
 0002:00000410       ??_C@_0FB@CKOMJLPB@jdk?1internal?1org?1jline?1terminal@ 0000000180004410     Kernel32.obj
 0002:00000468       ??_C@_0DO@KLOLFBPB@Ljdk?1internal?1org?1jline?1termina@ 0000000180004468     Kernel32.obj
 0002:000004a8       ??_C@_0BB@GCKPAHKE@dwCursorPosition@ 00000001800044a8     Kernel32.obj
 0002:000004c0       ??_C@_0M@LLNFGKPP@wAttributes@ 00000001800044c0     Kernel32.obj
 0002:000004d0       ??_C@_0ED@GDPBCFCF@Ljdk?1internal?1org?1jline?1termina@ 00000001800044d0     Kernel32.obj
 0002:00000518       ??_C@_08EGJHMBFD@srWindow@ 0000000180004518     Kernel32.obj
 0002:00000528       ??_C@_0BE@DLBDILN@dwMaximumWindowSize@ 0000000180004528     Kernel32.obj
 0002:00000540       ??_C@_0DM@IOLEMLOB@jdk?1internal?1org?1jline?1terminal@ 0000000180004540     Kernel32.obj
 0002:0000057c       ??_C@_01MMEEDKFM@X@        000000018000457c     Kernel32.obj
 0002:00000580       ??_C@_01NFFPALBN@Y@        0000000180004580     Kernel32.obj
 0002:00000590       ??_C@_0ED@KEABPHEC@jdk?1internal?1org?1jline?1terminal@ 0000000180004590     Kernel32.obj
 0002:000005d8       ??_C@_09KDLBEGCN@EventType@ 00000001800045d8     Kernel32.obj
 0002:000005f0       ??_C@_0FA@EPHOAIKB@Ljdk?1internal?1org?1jline?1termina@ 00000001800045f0     Kernel32.obj
 0002:00000640       ??_C@_05GCNIINAF@Event@    0000000180004640     Kernel32.obj
 0002:00000650       ??_C@_0EO@ENJPMKIB@jdk?1internal?1org?1jline?1terminal@ 0000000180004650     Kernel32.obj
 0002:000006a0       ??_C@_0EJ@KAFKPAON@Ljdk?1internal?1org?1jline?1termina@ 00000001800046a0     Kernel32.obj
 0002:000006f0       ??_C@_08IICPJOPF@KeyEvent@ 00000001800046f0     Kernel32.obj
 0002:00000700       ??_C@_0EL@NEMNNEIM@Ljdk?1internal?1org?1jline?1termina@ 0000000180004700     Kernel32.obj
 0002:00000750       ??_C@_0L@MEMIOFPE@MouseEvent@ 0000000180004750     Kernel32.obj
 0002:00000760       ??_C@_0FC@GJCMFPEB@Ljdk?1internal?1org?1jline?1termina@ 0000000180004760     Kernel32.obj
 0002:000007b8       ??_C@_0BG@FDJGLIMD@WindowBufferSizeEvent@ 00000001800047b8     Kernel32.obj
 0002:000007d0       ??_C@_0EK@GINBNDHB@Ljdk?1internal?1org?1jline?1termina@ 00000001800047d0     Kernel32.obj
 0002:00000820       ??_C@_09DGBBEBCO@MenuEvent@ 0000000180004820     Kernel32.obj
 0002:00000830       ??_C@_0EL@NEOCEPBL@Ljdk?1internal?1org?1jline?1termina@ 0000000180004830     Kernel32.obj
 0002:00000880       ??_C@_0L@PKFCPJDI@FocusEvent@ 0000000180004880     Kernel32.obj
 0002:00000890       ??_C@_0EH@LAMOGNLH@jdk?1internal?1org?1jline?1terminal@ 0000000180004890     Kernel32.obj
 0002:000008d8       ??_C@_08IOMBICKD@bKeyDown@ 00000001800048d8     Kernel32.obj
 0002:000008e8       ??_C@_0N@OFEBLKAO@wRepeatCount@ 00000001800048e8     Kernel32.obj
 0002:000008f8       ??_C@_0BA@ODMGPHEG@wVirtualKeyCode@ 00000001800048f8     Kernel32.obj
 0002:00000908       ??_C@_0BB@GLFALPCM@wVirtualScanCode@ 0000000180004908     Kernel32.obj
 0002:00000920       ??_C@_0BC@CPLAFJNJ@dwControlKeyState@ 0000000180004920     Kernel32.obj
 0002:00000940       ??_C@_0EJ@KJENNMFH@jdk?1internal?1org?1jline?1terminal@ 0000000180004940     Kernel32.obj
 0002:00000990       ??_C@_0BA@CLCFHGAI@dwMousePosition@ 0000000180004990     Kernel32.obj
 0002:000009a0       ??_C@_0O@OBJAOKMC@dwButtonState@ 00000001800049a0     Kernel32.obj
 0002:000009b0       ??_C@_0N@LGDKLHCN@dwEventFlags@ 00000001800049b0     Kernel32.obj
 0002:000009c0       ??_C@_0FA@ELBPHOIL@jdk?1internal?1org?1jline?1terminal@ 00000001800049c0     Kernel32.obj
 0002:00000a10       ??_C@_0EI@HEDGJHGB@jdk?1internal?1org?1jline?1terminal@ 0000000180004a10     Kernel32.obj
 0002:00000a58       ??_C@_0M@ILCOGF@dwCommandId@ 0000000180004a58     Kernel32.obj
 0002:00000a70       ??_C@_0EJ@IGNGELFH@jdk?1internal?1org?1jline?1terminal@ 0000000180004a70     Kernel32.obj
 0002:00000ac0       ??_C@_09LPEMLFBO@bSetFocus@ 0000000180004ac0     Kernel32.obj
 0002:00000ad0       ??_C@_0EB@FEHKODDE@jdk?1internal?1org?1jline?1terminal@ 0000000180004ad0     Kernel32.obj
 0002:00000b14       ??_C@_04KPCPLBPL@Left@     0000000180004b14     Kernel32.obj
 0002:00000b1c       ??_C@_03PGGAENPN@Top@      0000000180004b1c     Kernel32.obj
 0002:00000b20       ??_C@_05DADPALEM@Right@    0000000180004b20     Kernel32.obj
 0002:00000b28       ??_C@_06DDHCBBGN@Bottom@   0000000180004b28     Kernel32.obj
 0002:00000b30       ??_C@_0EA@CDONDDCN@jdk?1internal?1org?1jline?1terminal@ 0000000180004b30     Kernel32.obj
 0002:00000b70       ??_C@_01GFHCPBMG@C@        0000000180004b70     Kernel32.obj
 0002:00000b78       ??_C@_0M@PBJKDIHH@UnicodeChar@ 0000000180004b78     Kernel32.obj
 0002:00000b88       _pDefaultRawDllMain        0000000180004b88     MSVCRT:dll_dllmain.obj
 0002:00000b88       _pRawDllMain               0000000180004b88     MSVCRT:dll_dllmain.obj
 0002:00000ba0       __xmm@ffffffffffffffffffffffffffffffff 0000000180004ba0     MSVCRT:utility.obj
 0002:00000bb8       ??_7exception@std@@6B@     0000000180004bb8     MSVCRT:throw_bad_alloc.obj
 0002:00000bc8       ??_C@_0BC@EOODALEL@Unknown?5exception@ 0000000180004bc8     MSVCRT:throw_bad_alloc.obj
 0002:00000be8       ??_7bad_alloc@std@@6B@     0000000180004be8     MSVCRT:throw_bad_alloc.obj
 0002:00000bf8       ??_C@_0P@GHFPNOJB@bad?5allocation@ 0000000180004bf8     MSVCRT:throw_bad_alloc.obj
 0002:00000c10       ??_7bad_array_new_length@std@@6B@ 0000000180004c10     MSVCRT:throw_bad_alloc.obj
 0002:00000c20       ??_C@_0BF@KINCDENJ@bad?5array?5new?5length@ 0000000180004c20     MSVCRT:throw_bad_alloc.obj
 0002:00000c40       ??_7type_info@@6B@         0000000180004c40     MSVCRT:std_type_info_static.obj
 0002:00000c50       _load_config_used          0000000180004c50     MSVCRT:loadcfg.obj
 0002:00000e00       ??_R4exception@std@@6B@    0000000180004e00     MSVCRT:throw_bad_alloc.obj
 0002:00000e28       ??_R3exception@std@@8      0000000180004e28     MSVCRT:throw_bad_alloc.obj
 0002:00000e40       ??_R2exception@std@@8      0000000180004e40     MSVCRT:throw_bad_alloc.obj
 0002:00000e50       ??_R1A@?0A@EA@exception@std@@8 0000000180004e50     MSVCRT:throw_bad_alloc.obj
 0002:00000e78       ??_R4bad_alloc@std@@6B@    0000000180004e78     MSVCRT:throw_bad_alloc.obj
 0002:00000ea0       ??_R3bad_alloc@std@@8      0000000180004ea0     MSVCRT:throw_bad_alloc.obj
 0002:00000eb8       ??_R2bad_alloc@std@@8      0000000180004eb8     MSVCRT:throw_bad_alloc.obj
 0002:00000ed0       ??_R1A@?0A@EA@bad_alloc@std@@8 0000000180004ed0     MSVCRT:throw_bad_alloc.obj
 0002:00000ef8       ??_R4bad_array_new_length@std@@6B@ 0000000180004ef8     MSVCRT:throw_bad_alloc.obj
 0002:00000f20       ??_R3bad_array_new_length@std@@8 0000000180004f20     MSVCRT:throw_bad_alloc.obj
 0002:00000f38       ??_R2bad_array_new_length@std@@8 0000000180004f38     MSVCRT:throw_bad_alloc.obj
 0002:00000f58       ??_R1A@?0A@EA@bad_array_new_length@std@@8 0000000180004f58     MSVCRT:throw_bad_alloc.obj
 0002:00000f80       ??_R4type_info@@6B@        0000000180004f80     MSVCRT:std_type_info_static.obj
 0002:00000fa8       ??_R3type_info@@8          0000000180004fa8     MSVCRT:std_type_info_static.obj
 0002:00000fc0       ??_R2type_info@@8          0000000180004fc0     MSVCRT:std_type_info_static.obj
 0002:00000fd0       ??_R1A@?0A@EA@type_info@@8 0000000180004fd0     MSVCRT:std_type_info_static.obj
 0002:00000ff4       __volatile_metadata        0000000180004ff4     <linker-defined>
 0002:00001358       __rtc_iaa                  0000000180005358     MSVCRT:initsect.obj
 0002:00001360       __rtc_izz                  0000000180005360     MSVCRT:initsect.obj
 0002:00001368       __rtc_taa                  0000000180005368     MSVCRT:initsect.obj
 0002:00001370       __rtc_tzz                  0000000180005370     MSVCRT:initsect.obj
 0002:000015b8       _TI2?AVbad_alloc@std@@     00000001800055b8     MSVCRT:throw_bad_alloc.obj
 0002:000015d8       _CTA2?AVbad_alloc@std@@    00000001800055d8     MSVCRT:throw_bad_alloc.obj
 0002:000015f0       _CT??_R0?AVbad_alloc@std@@@8??0bad_alloc@std@@QEAA@AEBV01@@Z24 00000001800055f0     MSVCRT:throw_bad_alloc.obj
 0002:00001618       _CT??_R0?AVexception@std@@@8??0exception@std@@QEAA@AEBV01@@Z24 0000000180005618     MSVCRT:throw_bad_alloc.obj
 0002:00001640       _TI3?AVbad_array_new_length@std@@ 0000000180005640     MSVCRT:throw_bad_alloc.obj
 0002:00001660       _CTA3?AVbad_array_new_length@std@@ 0000000180005660     MSVCRT:throw_bad_alloc.obj
 0002:00001680       _CT??_R0?AVbad_array_new_length@std@@@8??0bad_array_new_length@std@@QEAA@AEBV01@@Z24 0000000180005680     MSVCRT:throw_bad_alloc.obj
 0002:00001bf0       __IMPORT_DESCRIPTOR_KERNEL32 0000000180005bf0     kernel32:KERNEL32.dll
 0002:00001c04       __IMPORT_DESCRIPTOR_VCRUNTIME140 0000000180005c04     vcruntime:VCRUNTIME140.dll
 0002:00001c18       __IMPORT_DESCRIPTOR_api-ms-win-crt-runtime-l1-1-0 0000000180005c18     ucrt:api-ms-win-crt-runtime-l1-1-0.dll
 0002:00001c2c       __IMPORT_DESCRIPTOR_api-ms-win-crt-heap-l1-1-0 0000000180005c2c     ucrt:api-ms-win-crt-heap-l1-1-0.dll
 0002:00001c40       __NULL_IMPORT_DESCRIPTOR   0000000180005c40     kernel32:KERNEL32.dll
 0003:00000000       __security_cookie_complement 0000000180007000     MSVCRT:gs_cookie.obj
 0003:00000008       __security_cookie          0000000180007008     MSVCRT:gs_cookie.obj
 0003:00000010       __scrt_native_dllmain_reason 0000000180007010     MSVCRT:utility.obj
 0003:00000018       __isa_available            0000000180007018     MSVCRT:cpu_disp.obj
 0003:0000001c       __isa_enabled              000000018000701c     MSVCRT:cpu_disp.obj
 0003:00000020       __memset_fast_string_threshold 0000000180007020     MSVCRT:cpu_disp.obj
 0003:00000028       __memset_nt_threshold      0000000180007028     MSVCRT:cpu_disp.obj
 0003:00000030       __scrt_ucrt_dll_is_in_use  0000000180007030     MSVCRT:ucrt_stubs.obj
 0003:00000038       ??_R0?AVbad_alloc@std@@@8  0000000180007038     MSVCRT:throw_bad_alloc.obj
 0003:00000060       ??_R0?AVexception@std@@@8  0000000180007060     MSVCRT:throw_bad_alloc.obj
 0003:00000088       ??_R0?AVbad_array_new_length@std@@@8 0000000180007088     MSVCRT:throw_bad_alloc.obj
 0003:000000b8       ??_R0?AVtype_info@@@8      00000001800070b8     MSVCRT:std_type_info_static.obj
 0003:00000880       ?__type_info_root_node@@3U__type_info_node@@A 0000000180007880     MSVCRT:tncleanup.obj
 0003:00000890       ?_OptionsStorage@?1??__local_stdio_printf_options@@9@4_KA 0000000180007890     MSVCRT:default_local_stdio_options.obj
 0003:00000898       ?_OptionsStorage@?1??__local_stdio_scanf_options@@9@4_KA 0000000180007898     MSVCRT:default_local_stdio_options.obj
 0003:000008a0       __scrt_current_native_startup_state 00000001800078a0     MSVCRT:utility.obj
 0003:000008a8       __scrt_native_startup_lock 00000001800078a8     MSVCRT:utility.obj
 0003:000008e8       __scrt_debugger_hook_flag  00000001800078e8     MSVCRT:utility_desktop.obj
 0003:000008ec       __favor                    00000001800078ec     MSVCRT:cpu_disp.obj
 0003:000008f0       __dyn_tls_init_callback    00000001800078f0     <common>

 entry point at        0001:00002040

 Static symbols

 0000:ffff5000       .debug$S                   0000000180000000     le.exp
 0000:ffff5000       .debug$S                   0000000180000000     vcruntime:VCRUNTIME140.dll
 0000:ffff5000       .debug$S                   0000000180000000     vcruntime:VCRUNTIME140.dll
 0000:ffff5000       .debug$S                   0000000180000000     vcruntime:VCRUNTIME140.dll
 0000:ffff5000       .debug$S                   0000000180000000     vcruntime:VCRUNTIME140.dll
 0000:ffff5000       .debug$S                   0000000180000000     vcruntime:VCRUNTIME140.dll
 0000:ffff5000       .debug$S                   0000000180000000     vcruntime:VCRUNTIME140.dll
 0000:ffff5000       .debug$S                   0000000180000000     vcruntime:VCRUNTIME140.dll
 0000:ffff5000       .debug$S                   0000000180000000     vcruntime:VCRUNTIME140.dll
 0000:ffff5000       .debug$S                   0000000180000000     vcruntime:VCRUNTIME140.dll
 0000:ffff5000       .debug$S                   0000000180000000     ucrt:api-ms-win-crt-heap-l1-1-0.dll
 0000:ffff5000       .debug$S                   0000000180000000     ucrt:api-ms-win-crt-heap-l1-1-0.dll
 0000:ffff5000       .debug$S                   0000000180000000     ucrt:api-ms-win-crt-heap-l1-1-0.dll
 0000:ffff5000       .debug$S                   0000000180000000     ucrt:api-ms-win-crt-runtime-l1-1-0.dll
 0000:ffff5000       .debug$S                   0000000180000000     ucrt:api-ms-win-crt-runtime-l1-1-0.dll
 0000:ffff5000       .debug$S                   0000000180000000     ucrt:api-ms-win-crt-runtime-l1-1-0.dll
 0000:ffff5000       .debug$S                   0000000180000000     ucrt:api-ms-win-crt-runtime-l1-1-0.dll
 0000:ffff5000       .debug$S                   0000000180000000     ucrt:api-ms-win-crt-runtime-l1-1-0.dll
 0000:ffff5000       .debug$S                   0000000180000000     ucrt:api-ms-win-crt-runtime-l1-1-0.dll
 0000:ffff5000       .debug$S                   0000000180000000     ucrt:api-ms-win-crt-runtime-l1-1-0.dll
 0000:ffff5000       .debug$S                   0000000180000000     ucrt:api-ms-win-crt-runtime-l1-1-0.dll
 0000:ffff5000       .debug$S                   0000000180000000     ucrt:api-ms-win-crt-runtime-l1-1-0.dll
 0000:ffff5000       .debug$S                   0000000180000000     ucrt:api-ms-win-crt-runtime-l1-1-0.dll
 0000:ffff5000       .debug$S                   0000000180000000     ucrt:api-ms-win-crt-runtime-l1-1-0.dll
 0000:ffff5000       .debug$S                   0000000180000000     ucrt:api-ms-win-crt-runtime-l1-1-0.dll
 0000:ffff5000       .debug$S                   0000000180000000     kernel32:KERNEL32.dll
 0000:ffff5000       .debug$S                   0000000180000000     kernel32:KERNEL32.dll
 0000:ffff5000       .debug$S                   0000000180000000     kernel32:KERNEL32.dll
 0000:ffff5000       .debug$S                   0000000180000000     kernel32:KERNEL32.dll
 0000:ffff5000       .debug$S                   0000000180000000     kernel32:KERNEL32.dll
 0000:ffff5000       .debug$S                   0000000180000000     kernel32:KERNEL32.dll
 0000:ffff5000       .debug$S                   0000000180000000     kernel32:KERNEL32.dll
 0000:ffff5000       .debug$S                   0000000180000000     kernel32:KERNEL32.dll
 0000:ffff5000       .debug$S                   0000000180000000     kernel32:KERNEL32.dll
 0000:ffff5000       .debug$S                   0000000180000000     kernel32:KERNEL32.dll
 0000:ffff5000       .debug$S                   0000000180000000     kernel32:KERNEL32.dll
 0000:ffff5000       .debug$S                   0000000180000000     kernel32:KERNEL32.dll
 0000:ffff5000       .debug$S                   0000000180000000     kernel32:KERNEL32.dll
 0000:ffff5000       .debug$S                   0000000180000000     kernel32:KERNEL32.dll
 0000:ffff5000       .debug$S                   0000000180000000     kernel32:KERNEL32.dll
 0000:ffff5000       .debug$S                   0000000180000000     kernel32:KERNEL32.dll
 0000:ffff5000       .debug$S                   0000000180000000     kernel32:KERNEL32.dll
 0000:ffff5000       .debug$S                   0000000180000000     kernel32:KERNEL32.dll
 0000:ffff5000       .debug$S                   0000000180000000     kernel32:KERNEL32.dll
 0000:ffff5000       .debug$S                   0000000180000000     kernel32:KERNEL32.dll
 0000:ffff5000       .debug$S                   0000000180000000     kernel32:KERNEL32.dll
 0000:ffff5000       .debug$S                   0000000180000000     kernel32:KERNEL32.dll
 0000:ffff5000       .debug$S                   0000000180000000     kernel32:KERNEL32.dll
 0000:ffff5000       .debug$S                   0000000180000000     kernel32:KERNEL32.dll
 0000:ffff5000       .debug$S                   0000000180000000     kernel32:KERNEL32.dll
 0000:ffff5000       .debug$S                   0000000180000000     kernel32:KERNEL32.dll
 0000:ffff5000       .debug$S                   0000000180000000     kernel32:KERNEL32.dll
 0000:ffff5000       .debug$S                   0000000180000000     kernel32:KERNEL32.dll
 0000:ffff5000       .debug$S                   0000000180000000     kernel32:KERNEL32.dll
 0000:ffff5000       .debug$S                   0000000180000000     kernel32:KERNEL32.dll
 0000:ffff5000       .debug$S                   0000000180000000     kernel32:KERNEL32.dll
 0001:00001cf0       $$000000                   0000000180002cf0     MSVCRT:amdsecgs.obj
 0001:00001d20       ?dllmain_crt_dispatch@@YAHQEAUHINSTANCE__@@KQEAX@Z 0000000180002d20 f   MSVCRT:dll_dllmain.obj
 0001:00001d70       ?dllmain_crt_process_attach@@YAHQEAUHINSTANCE__@@QEAX@Z 0000000180002d70 f   MSVCRT:dll_dllmain.obj
 0001:00001e88       ?dllmain_crt_process_detach@@YAH_N@Z 0000000180002e88 f   MSVCRT:dll_dllmain.obj
 0001:00001f0c       ?dllmain_dispatch@@YAHQEAUHINSTANCE__@@KQEAX@Z 0000000180002f0c f   MSVCRT:dll_dllmain.obj
 0001:000021cc       capture_previous_context   00000001800031cc f   MSVCRT:gs_report.obj
 0001:00002c70       $$000000                   0000000180003c70     MSVCRT:guard_dispatch.obj
 0001:00002c90       $$000000                   0000000180003c90     MSVCRT:guard_xfg_dispatch.obj
 0001:00002ca6       ?fin$0@?0??dllmain_crt_process_attach@@YAHQEAUHINSTANCE__@@QEAX@Z@4HA 0000000180003ca6 f   MSVCRT:dll_dllmain.obj
 0001:00002cbd       ?fin$0@?0??dllmain_crt_process_detach@@YAH_N@Z@4HA 0000000180003cbd f   MSVCRT:dll_dllmain.obj
 0001:00002cd6       ?fin$1@?0??dllmain_crt_process_detach@@YAH_N@Z@4HA 0000000180003cd6 f   MSVCRT:dll_dllmain.obj
 0001:00002cea       ?filt$0@?0??dllmain_dispatch@@YAHQEAUHINSTANCE__@@KQEAX@Z@4HA 0000000180003cea f   MSVCRT:dll_dllmain.obj
 0001:00002d20       __scrt_is_nonwritable_in_current_image$filt$0 0000000180003d20 f   MSVCRT:utility.obj
 0002:00000b90       GS_ExceptionPointers       0000000180004b90     MSVCRT:gs_report.obj
 0002:00001378       $unwind$?NewObject@JNIEnv_@@QEAAPEAV_jobject@@PEAV_jclass@@PEAU_jmethodID@@ZZ 0000000180005378     Kernel32.obj
 0002:00001380       $unwind$Java_jdk_internal_org_jline_terminal_impl_jna_win_Kernel32Impl_initIDs 0000000180005380     Kernel32.obj
 0002:0000139c       $unwind$Java_jdk_internal_org_jline_terminal_impl_jna_win_Kernel32Impl_WaitForSingleObject 000000018000539c     Kernel32.obj
 0002:0000139c       $unwind$__raise_securityfailure 000000018000539c     MSVCRT:gs_report.obj
 0002:0000139c       $unwind$??2@YAPEAX_K@Z     000000018000539c     MSVCRT:new_scalar.obj
 0002:0000139c       $unwind$??_Gtype_info@@UEAAPEAXI@Z 000000018000539c     MSVCRT:std_type_info_static.obj
 0002:0000139c       $unwind$??0bad_alloc@std@@QEAA@AEBV01@@Z 000000018000539c     MSVCRT:throw_bad_alloc.obj
 0002:0000139c       $unwind$??0bad_array_new_length@std@@QEAA@AEBV01@@Z 000000018000539c     MSVCRT:throw_bad_alloc.obj
 0002:0000139c       $unwind$??0exception@std@@QEAA@AEBV01@@Z 000000018000539c     MSVCRT:throw_bad_alloc.obj
 0002:0000139c       $unwind$__scrt_initialize_crt 000000018000539c     MSVCRT:utility.obj
 0002:0000139c       $unwind$__scrt_initialize_onexit_tables 000000018000539c     MSVCRT:utility.obj
 0002:0000139c       $unwind$__scrt_release_startup_lock 000000018000539c     MSVCRT:utility.obj
 0002:0000139c       $unwind$__scrt_uninitialize_crt 000000018000539c     MSVCRT:utility.obj
 0002:000013a4       $unwind$Java_jdk_internal_org_jline_terminal_impl_jna_win_Kernel32Impl_FillConsoleOutputAttribute 00000001800053a4     Kernel32.obj
 0002:000013a4       $unwind$Java_jdk_internal_org_jline_terminal_impl_jna_win_Kernel32Impl_FillConsoleOutputCharacter 00000001800053a4     Kernel32.obj
 0002:000013b4       $unwind$Java_jdk_internal_org_jline_terminal_impl_jna_win_Kernel32Impl_GetConsoleMode 00000001800053b4     Kernel32.obj
 0002:000013c0       $unwind$Java_jdk_internal_org_jline_terminal_impl_jna_win_Kernel32Impl_GetConsoleScreenBufferInfo 00000001800053c0     Kernel32.obj
 0002:000013d8       $unwind$Java_jdk_internal_org_jline_terminal_impl_jna_win_Kernel32Impl_ReadConsoleInput 00000001800053d8     Kernel32.obj
 0002:000013f4       $unwind$Java_jdk_internal_org_jline_terminal_impl_jna_win_Kernel32Impl_SetConsoleCursorPosition 00000001800053f4     Kernel32.obj
 0002:00001404       $unwind$Java_jdk_internal_org_jline_terminal_impl_jna_win_Kernel32Impl_SetConsoleMode 0000000180005404     Kernel32.obj
 0002:00001404       $unwind$Java_jdk_internal_org_jline_terminal_impl_jna_win_Kernel32Impl_SetConsoleTextAttribute 0000000180005404     Kernel32.obj
 0002:00001404       $unwind$_RTC_Initialize    0000000180005404     MSVCRT:initsect.obj
 0002:00001404       $unwind$_RTC_Terminate     0000000180005404     MSVCRT:initsect.obj
 0002:00001404       $unwind$??_Gbad_alloc@std@@UEAAPEAXI@Z 0000000180005404     MSVCRT:throw_bad_alloc.obj
 0002:00001404       $unwind$??_Gbad_array_new_length@std@@UEAAPEAXI@Z 0000000180005404     MSVCRT:throw_bad_alloc.obj
 0002:00001404       $unwind$??_Gexception@std@@UEAAPEAXI@Z 0000000180005404     MSVCRT:throw_bad_alloc.obj
 0002:00001410       $unwind$Java_jdk_internal_org_jline_terminal_impl_jna_win_Kernel32Impl_SetConsoleTitle 0000000180005410     Kernel32.obj
 0002:00001410       $unwind$_DllMainCRTStartup 0000000180005410     MSVCRT:dll_dllmain.obj
 0002:00001420       $unwind$Java_jdk_internal_org_jline_terminal_impl_jna_win_Kernel32Impl_WriteConsoleW 0000000180005420     Kernel32.obj
 0002:00001434       $unwind$Java_jdk_internal_org_jline_terminal_impl_jna_win_Kernel32Impl_ScrollConsoleScreenBuffer 0000000180005434     Kernel32.obj
 0002:00001448       $unwind$__GSHandlerCheckCommon 0000000180005448     MSVCRT:gshandler.obj
 0002:00001450       $unwind$__scrt_initialize_default_local_stdio_options 0000000180005450     MSVCRT:default_local_stdio_options.obj
 0002:00001450       $unwind$?dllmain_crt_dispatch@@YAHQEAUHINSTANCE__@@KQEAX@Z 0000000180005450     MSVCRT:dll_dllmain.obj
 0002:00001450       $unwind$DllMain            0000000180005450     MSVCRT:dll_dllmain_stub.obj
 0002:00001450       $unwind$__GSHandlerCheck   0000000180005450     MSVCRT:gshandler.obj
 0002:00001450       $unwind$__scrt_acquire_startup_lock 0000000180005450     MSVCRT:utility.obj
 0002:00001450       $unwind$__scrt_dllmain_after_initialize_c 0000000180005450     MSVCRT:utility.obj
 0002:00001450       $unwind$__scrt_dllmain_before_initialize_c 0000000180005450     MSVCRT:utility.obj
 0002:00001450       $unwind$__scrt_dllmain_crt_thread_attach 0000000180005450     MSVCRT:utility.obj
 0002:00001450       $unwind$__scrt_dllmain_crt_thread_detach 0000000180005450     MSVCRT:utility.obj
 0002:00001450       $unwind$__scrt_dllmain_uninitialize_c 0000000180005450     MSVCRT:utility.obj
 0002:00001450       $unwind$__scrt_dllmain_uninitialize_critical 0000000180005450     MSVCRT:utility.obj
 0002:00001458       $xdatasym                  0000000180005458     MSVCRT:amdsecgs.obj
 0002:0000145c       $unwind$?dllmain_crt_process_attach@@YAHQEAUHINSTANCE__@@QEAX@Z 000000018000545c     MSVCRT:dll_dllmain.obj
 0002:00001498       $unwind$?fin$0@?0??dllmain_crt_process_attach@@YAHQEAUHINSTANCE__@@QEAX@Z@4HA 0000000180005498     MSVCRT:dll_dllmain.obj
 0002:00001498       $unwind$?fin$0@?0??dllmain_crt_process_detach@@YAH_N@Z@4HA 0000000180005498     MSVCRT:dll_dllmain.obj
 0002:00001498       $unwind$?fin$1@?0??dllmain_crt_process_detach@@YAH_N@Z@4HA 0000000180005498     MSVCRT:dll_dllmain.obj
 0002:000014a0       $unwind$?dllmain_crt_process_detach@@YAH_N@Z 00000001800054a0     MSVCRT:dll_dllmain.obj
 0002:000014f4       $unwind$?dllmain_dispatch@@YAHQEAUHINSTANCE__@@KQEAX@Z 00000001800054f4     MSVCRT:dll_dllmain.obj
 0002:0000151c       $unwind$?filt$0@?0??dllmain_dispatch@@YAHQEAUHINSTANCE__@@KQEAX@Z@4HA 000000018000551c     MSVCRT:dll_dllmain.obj
 0002:00001524       $unwind$__report_gsfailure 0000000180005524     MSVCRT:gs_report.obj
 0002:0000152c       $unwind$capture_previous_context 000000018000552c     MSVCRT:gs_report.obj
 0002:00001538       $unwind$__security_init_cookie 0000000180005538     MSVCRT:gs_support.obj
 0002:00001544       $unwind$__scrt_is_nonwritable_in_current_image 0000000180005544     MSVCRT:utility.obj
 0002:00001564       $unwind$__scrt_is_nonwritable_in_current_image$filt$0 0000000180005564     MSVCRT:utility.obj
 0002:0000156c       $unwind$__scrt_dllmain_exception_filter 000000018000556c     MSVCRT:utility.obj
 0002:00001580       $unwind$__scrt_fastfail    0000000180005580     MSVCRT:utility_desktop.obj
 0002:00001590       $unwind$?__scrt_throw_std_bad_alloc@@YAXXZ 0000000180005590     MSVCRT:throw_bad_alloc.obj
 0002:00001590       $unwind$?__scrt_throw_std_bad_array_new_length@@YAXXZ 0000000180005590     MSVCRT:throw_bad_alloc.obj
 0002:00001598       $unwind$__isa_available_init 0000000180005598     MSVCRT:cpu_disp.obj
 0002:000015a8       $xdatasym                  00000001800055a8     MSVCRT:guard_dispatch.obj
 0002:000015b0       $xdatasym                  00000001800055b0     MSVCRT:guard_xfg_dispatch.obj
 0002:000016b0       .edata                     00000001800056b0     le.exp
 0002:000016d8       rgpv                       00000001800056d8     le.exp
 0002:00001710       rgszName                   0000000180005710     le.exp
 0002:00001748       rgwOrd                     0000000180005748     le.exp
 0002:00001764       szName                     0000000180005764     le.exp
 0002:0000176b       $N00001                    000000018000576b     le.exp
 0002:000017c5       $N00002                    00000001800057c5     le.exp
 0002:0000181f       $N00003                    000000018000581f     le.exp
 0002:0000186d       $N00004                    000000018000586d     le.exp
 0002:000018c7       $N00005                    00000001800058c7     le.exp
 0002:00001913       $N00006                    0000000180005913     le.exp
 0002:00001963       $N00007                    0000000180005963     le.exp
 0002:000019bc       $N00008                    00000001800059bc     le.exp
 0002:00001a14       $N00009                    0000000180005a14     le.exp
 0002:00001a62       $N00010                    0000000180005a62     le.exp
 0002:00001ab9       $N00011                    0000000180005ab9     le.exp
 0002:00001b08       $N00012                    0000000180005b08     le.exp
 0002:00001b5b       $N00013                    0000000180005b5b     le.exp
 0002:00001ba8       $N00014                    0000000180005ba8     le.exp
 0002:00002096       .idata$6                   0000000180006096     kernel32:KERNEL32.dll
 0002:0000212e       .idata$6                   000000018000612e     vcruntime:VCRUNTIME140.dll
 0002:00002204       .idata$6                   0000000180006204     ucrt:api-ms-win-crt-runtime-l1-1-0.dll
 0002:00002226       .idata$6                   0000000180006226     ucrt:api-ms-win-crt-heap-l1-1-0.dll
 0003:000000e0       ?pointerClass@@3PEAV_jclass@@EA 00000001800070e0     Kernel32.obj
 0003:000000e8       ?pointerConstructor@@3PEAU_jmethodID@@EA 00000001800070e8     Kernel32.obj
 0003:000000f0       ?pointerValue@@3PEAU_jfieldID@@EA 00000001800070f0     Kernel32.obj
 0003:000000f8       ?intByReferenceClass@@3PEAV_jclass@@EA 00000001800070f8     Kernel32.obj
 0003:00000100       ?intByReferenceValue@@3PEAU_jfieldID@@EA 0000000180007100     Kernel32.obj
 0003:00000108       ?lastErrorExceptionClass@@3PEAV_jclass@@EA 0000000180007108     Kernel32.obj
 0003:00000110       ?lastErrorExceptionConstructor@@3PEAU_jmethodID@@EA 0000000180007110     Kernel32.obj
 0003:00000118       ?CHAR_INFO_Class@@3PEAV_jclass@@EA 0000000180007118     Kernel32.obj
 0003:00000120       ?CHAR_INFO_Constructor@@3PEAU_jmethodID@@EA 0000000180007120     Kernel32.obj
 0003:00000128       ?CHAR_INFO_uChar@@3PEAU_jfieldID@@EA 0000000180007128     Kernel32.obj
 0003:00000130       ?CHAR_INFO_Attributes@@3PEAU_jfieldID@@EA 0000000180007130     Kernel32.obj
 0003:00000138       ?CONSOLE_CURSOR_INFO_Class@@3PEAV_jclass@@EA 0000000180007138     Kernel32.obj
 0003:00000140       ?CONSOLE_CURSOR_INFO_Constructor@@3PEAU_jmethodID@@EA 0000000180007140     Kernel32.obj
 0003:00000148       ?CONSOLE_CURSOR_INFO_dwSize@@3PEAU_jfieldID@@EA 0000000180007148     Kernel32.obj
 0003:00000150       ?CONSOLE_CURSOR_INFO_bVisible@@3PEAU_jfieldID@@EA 0000000180007150     Kernel32.obj
 0003:00000158       ?CONSOLE_SCREEN_BUFFER_INFO_Class@@3PEAV_jclass@@EA 0000000180007158     Kernel32.obj
 0003:00000160       ?CONSOLE_SCREEN_BUFFER_INFO_Constructor@@3PEAU_jmethodID@@EA 0000000180007160     Kernel32.obj
 0003:00000168       ?CONSOLE_SCREEN_BUFFER_INFO_dwSize@@3PEAU_jfieldID@@EA 0000000180007168     Kernel32.obj
 0003:00000170       ?CONSOLE_SCREEN_BUFFER_INFO_dwCursorPosition@@3PEAU_jfieldID@@EA 0000000180007170     Kernel32.obj
 0003:00000178       ?CONSOLE_SCREEN_BUFFER_INFO_wAttributes@@3PEAU_jfieldID@@EA 0000000180007178     Kernel32.obj
 0003:00000180       ?CONSOLE_SCREEN_BUFFER_INFO_srWindow@@3PEAU_jfieldID@@EA 0000000180007180     Kernel32.obj
 0003:00000188       ?CONSOLE_SCREEN_BUFFER_INFO_dwMaximumWindowSize@@3PEAU_jfieldID@@EA 0000000180007188     Kernel32.obj
 0003:00000190       ?COORD_Class@@3PEAV_jclass@@EA 0000000180007190     Kernel32.obj
 0003:00000198       ?COORD_Constructor@@3PEAU_jmethodID@@EA 0000000180007198     Kernel32.obj
 0003:000001a0       ?COORD_X@@3PEAU_jfieldID@@EA 00000001800071a0     Kernel32.obj
 0003:000001a8       ?COORD_Y@@3PEAU_jfieldID@@EA 00000001800071a8     Kernel32.obj
 0003:000001b0       ?INPUT_RECORD_Class@@3PEAV_jclass@@EA 00000001800071b0     Kernel32.obj
 0003:000001b8       ?INPUT_RECORD_Constructor@@3PEAU_jmethodID@@EA 00000001800071b8     Kernel32.obj
 0003:000001c0       ?INPUT_RECORD_EventType@@3PEAU_jfieldID@@EA 00000001800071c0     Kernel32.obj
 0003:000001c8       ?INPUT_RECORD_Event@@3PEAU_jfieldID@@EA 00000001800071c8     Kernel32.obj
 0003:000001d0       ?EventUnion_Class@@3PEAV_jclass@@EA 00000001800071d0     Kernel32.obj
 0003:000001d8       ?EventUnion_Constructor@@3PEAU_jmethodID@@EA 00000001800071d8     Kernel32.obj
 0003:000001e0       ?EventUnion_KeyEvent@@3PEAU_jfieldID@@EA 00000001800071e0     Kernel32.obj
 0003:000001e8       ?EventUnion_MouseEvent@@3PEAU_jfieldID@@EA 00000001800071e8     Kernel32.obj
 0003:000001f0       ?EventUnion_WindowBufferSizeEvent@@3PEAU_jfieldID@@EA 00000001800071f0     Kernel32.obj
 0003:000001f8       ?EventUnion_MenuEvent@@3PEAU_jfieldID@@EA 00000001800071f8     Kernel32.obj
 0003:00000200       ?EventUnion_FocusEvent@@3PEAU_jfieldID@@EA 0000000180007200     Kernel32.obj
 0003:00000208       ?KEY_EVENT_RECORD_Class@@3PEAV_jclass@@EA 0000000180007208     Kernel32.obj
 0003:00000210       ?KEY_EVENT_RECORD_Constructor@@3PEAU_jmethodID@@EA 0000000180007210     Kernel32.obj
 0003:00000218       ?KEY_EVENT_RECORD_bKeyDown@@3PEAU_jfieldID@@EA 0000000180007218     Kernel32.obj
 0003:00000220       ?KEY_EVENT_RECORD_wRepeatCount@@3PEAU_jfieldID@@EA 0000000180007220     Kernel32.obj
 0003:00000228       ?KEY_EVENT_RECORD_wVirtualKeyCode@@3PEAU_jfieldID@@EA 0000000180007228     Kernel32.obj
 0003:00000230       ?KEY_EVENT_RECORD_wVirtualScanCode@@3PEAU_jfieldID@@EA 0000000180007230     Kernel32.obj
 0003:00000238       ?KEY_EVENT_RECORD_uChar@@3PEAU_jfieldID@@EA 0000000180007238     Kernel32.obj
 0003:00000240       ?KEY_EVENT_RECORD_dwControlKeyState@@3PEAU_jfieldID@@EA 0000000180007240     Kernel32.obj
 0003:00000248       ?MOUSE_EVENT_RECORD_Class@@3PEAV_jclass@@EA 0000000180007248     Kernel32.obj
 0003:00000250       ?MOUSE_EVENT_RECORD_Constructor@@3PEAU_jmethodID@@EA 0000000180007250     Kernel32.obj
 0003:00000258       ?MOUSE_EVENT_RECORD_dwMousePosition@@3PEAU_jfieldID@@EA 0000000180007258     Kernel32.obj
 0003:00000260       ?MOUSE_EVENT_RECORD_dwButtonState@@3PEAU_jfieldID@@EA 0000000180007260     Kernel32.obj
 0003:00000268       ?MOUSE_EVENT_RECORD_dwControlKeyState@@3PEAU_jfieldID@@EA 0000000180007268     Kernel32.obj
 0003:00000270       ?MOUSE_EVENT_RECORD_dwEventFlags@@3PEAU_jfieldID@@EA 0000000180007270     Kernel32.obj
 0003:00000278       ?WINDOW_BUFFER_SIZE_RECORD_Class@@3PEAV_jclass@@EA 0000000180007278     Kernel32.obj
 0003:00000280       ?WINDOW_BUFFER_SIZE_RECORD_Constructor@@3PEAU_jmethodID@@EA 0000000180007280     Kernel32.obj
 0003:00000288       ?WINDOW_BUFFER_SIZE_RECORD_dwSize@@3PEAU_jfieldID@@EA 0000000180007288     Kernel32.obj
 0003:00000290       ?MENU_EVENT_RECORD_Class@@3PEAV_jclass@@EA 0000000180007290     Kernel32.obj
 0003:00000298       ?MENU_EVENT_RECORD_Constructor@@3PEAU_jmethodID@@EA 0000000180007298     Kernel32.obj
 0003:000002a0       ?MENU_EVENT_RECORD_dwCommandId@@3PEAU_jfieldID@@EA 00000001800072a0     Kernel32.obj
 0003:000002a8       ?FOCUS_EVENT_RECORD_Class@@3PEAV_jclass@@EA 00000001800072a8     Kernel32.obj
 0003:000002b0       ?FOCUS_EVENT_RECORD_Constructor@@3PEAU_jmethodID@@EA 00000001800072b0     Kernel32.obj
 0003:000002b8       ?FOCUS_EVENT_RECORD_bSetFocus@@3PEAU_jfieldID@@EA 00000001800072b8     Kernel32.obj
 0003:000002c0       ?SMALL_RECT_Class@@3PEAV_jclass@@EA 00000001800072c0     Kernel32.obj
 0003:000002c8       ?SMALL_RECT_Constructor@@3PEAU_jmethodID@@EA 00000001800072c8     Kernel32.obj
 0003:000002d0       ?SMALL_RECT_Left@@3PEAU_jfieldID@@EA 00000001800072d0     Kernel32.obj
 0003:000002d8       ?SMALL_RECT_Top@@3PEAU_jfieldID@@EA 00000001800072d8     Kernel32.obj
 0003:000002e0       ?SMALL_RECT_Right@@3PEAU_jfieldID@@EA 00000001800072e0     Kernel32.obj
 0003:000002e8       ?SMALL_RECT_Bottom@@3PEAU_jfieldID@@EA 00000001800072e8     Kernel32.obj
 0003:000002f0       ?UnionChar_Class@@3PEAV_jclass@@EA 00000001800072f0     Kernel32.obj
 0003:000002f8       ?UnionChar_Constructor@@3PEAU_jmethodID@@EA 00000001800072f8     Kernel32.obj
 0003:00000300       ?UnionChar_UnicodeChar@@3PEAU_jfieldID@@EA 0000000180007300     Kernel32.obj
 0003:00000308       ?__proc_attached@@3HA      0000000180007308     MSVCRT:dll_dllmain.obj
 0003:00000310       GS_ExceptionRecord         0000000180007310     MSVCRT:gs_report.obj
 0003:000003b0       GS_ContextRecord           00000001800073b0     MSVCRT:gs_report.obj
 0003:000008b0       ?is_initialized_as_dll@@3_NA 00000001800078b0     MSVCRT:utility.obj
 0003:000008b1       ?module_local_atexit_table_initialized@@3_NA 00000001800078b1     MSVCRT:utility.obj
 0003:000008b8       ?module_local_atexit_table@@3U_onexit_table_t@@A 00000001800078b8     MSVCRT:utility.obj
 0003:000008d0       ?module_local_at_quick_exit_table@@3U_onexit_table_t@@A 00000001800078d0     MSVCRT:utility.obj
 0005:00000060       $R000000                   0000000180009060     le.dll.res
